:04000000F1EF06F026
:08000800046ED8CF05F0E0CF33
:1000100006F00001E9CF0CF0EACF07F0E1CF08F0DD
:10002000E2CF09F0D9CF0AF0DACF0BF0F3CF12F01C
:10003000F4CF13F0FACF14F0F5CF15F0F6CF16F099
:10004000F7CF17F000C00EF001C00FF002C010F0A3
:1000500003C011F09DA030EF00F09EB0F8EF02F069
:100060009DA236EF00F09EB20BEF03F09DAA3CEF8D
:1000700000F09EBA2DEF03F09DA842EF00F09EB86D
:1000800062EF03F00EC000F00FC001F010C002F0EC
:1000900011C003F00CC0E9FF07C0EAFF078E08C0DB
:1000A000E1FF09C0E2FF0AC0D9FF0BC0DAFF12C0AE
:1000B000F3FF13C0F4FF14C0FAFF15C0F5FF16C01C
:1000C000F6FF17C0F7FF045006C0E0FF05C0D8FFD9
:1000D0001000E00FF66E000EF7220900F550120036
:1000E00000000000000000000000000000183C3C80
:1000F0003C18180018180000006666660000000032
:10010000000000000036367F3636367F3636000077
:10011000083E6B68683E0B0B6B3E080870D8DA76B9
:100120000C18306E5B1B0E0000386C6C386CC7C648
:100130006E3B0000001818180000000000000000CE
:10014000000C1818303030303018180C00301818E7
:100150000C0C0C0C0C181830000000361C7F1C36E0
:100160000000000000000018187E181800000000B1
:10017000000000000000000018183000000000001F
:10018000007E0000000000000000000000000000F1
:10019000181800000006060C0C18183030606000BB
:1001A000001C36636B6B6B63361C0000000C1C3C40
:1001B0000C0C0C0C0C3F0000003C6606060C1830C2
:1001C000607E0000003C6666061C0666663C000019
:1001D00000060E1E3666667F06060000007E606022
:1001E000607C0606663C0000001C3060607C666631
:1001F000663C0000007E060C0C1818181818000049
:10020000003C6666663C6666663C0000003C6666CE
:10021000663E06060C3800000000001818000000BA
:10022000181800000000001818000000181830000E
:1002300000060C18306030180C06000000000000AA
:100240007E007E0000000000006030180C060C18D4
:1002500030600000003C66660C181800181800009A
:10026000007EC3C3CFDBDBCFC07F000000183C663D
:1002700066667E6666660000007C6666667C66660C
:10028000667C0000003C666060606060663C000068
:1002900000786C66666666666C780000007E60605A
:1002A000607C6060607E0000007E6060607C6060FA
:1002B00060600000003C666060606E66663E000044
:1002C00000666666667E666666660000003C181814
:1002D00018181818183C00000006060606060666E0
:1002E000663C00000066666C6C786C6C66660000AC
:1002F0000060606060606060607E00000063777F27
:100300006B6B636363630000006363737B6F67639E
:1003100063630000003C666666666666663C0000D5
:10032000007C6666667C606060600000003C66661B
:1003300066666666663C0C06007C6666667C6C6675
:1003400066660000003C666030180C06663C0000E3
:10035000007E18181818181818180000006666662D
:1003600066666666663C0000006666666666666689
:100370003C18000000636363636B6B6B3E360000E8
:10038000006666663C183C66666600000066666647
:10039000663C181818180000007E06060C1830601D
:1003A000607E00003C303030303030303030303C17
:1003B000006060303018180C0C0606003C0C0C0C69
:1003C0000C0C0C0C0C0C0C3C183C660000000000E3
:1003D000000000000000000000000000000000FF1E
:1003E0003030180000000000000000000000003C59
:1003F00006063E66663E00000060607C66666666D5
:10040000667C00000000003C66606060663C0000A6
:100410000006063E66666666663E00000000003C1A
:1004200066667E60603C0000001C30303078303002
:10043000303000000000003E66666666663E063CA0
:100440000060607C66666666666600001818007864
:1004500018181818187E00000C0C003C0C0C0C0C22
:100460000C0C0C7800606066666C786C6666000048
:100470000078181818181818187E00000000007E60
:100480006B6B6B6B6B6300000000007C66666666DE
:10049000666600000000003C66666666663C00001A
:1004A0000000007C66666666667C60600000003E58
:1004B00066666666663E06060000007C66606060F2
:1004C000606000000000003E60603C06067C0000AA
:1004D0000030307830303030301C000000000066D2
:1004E00066666666663E00000000006666666666D2
:1004F0003C1800000000006363636B6B3E36000035
:1005000000000066663C183C66660000000000665D
:1005100066666666663E067C0000007E060C183045
:10052000607E0000C0C0C0C0C0C0C0C0C0C0C0C0ED
:1005300018181818180018181818180003030303BF
:1005400003030303030303030076DC000000000041
:1005500000000000001818003C063E66663E0000E1
:10056000002424003C063E66663E00000024240071
:100570003C666666663C00001818003C66667E664F
:10058000666600002424003C66667E66666600009F
:100590002424003C66666666663C00000000183C49
:1005A0007EFF181818180000000018181818FF7E91
:1005B0003C1800000000080C0EFFFF0E0C080000A5
:1005C0000000103070FFFF70301000003C66663C89
:1005D0000000000000000000F76AE80FF66E050E4C
:1005E000F7220900F5501200010204081020408093
:1005F000DC0ECF6ECE6A04000401252B2551640861
:1006000002E1256B1A839E90000142EF00F09EA844
:10061000FED7AD6E1200BA94ABA80CD0AB9882880E
:1006200004011B510001F3DF010E0401236F9D88BB
:1006300004D000018298AB8804019E92000142EF31
:1006400000F09EAAFED7ABCF19F0AECF01F019A2F1
:1006500002D0AB98AB882EEF03F0F3D701C073F450
:1006600004017351010A000103E0030A04E018D0F9
:100670000401246B23D00401245112080FE12651F8
:100680001F0B04080BE126AF02D01A8501D01A9582
:1006900026AD02D0808601D08096BA840FD00001AA
:1006A0000401245111080AE32451242B036A260F64
:1006B000E96E040E0320EA6E73C4EFFF9E9A0001F8
:1006C00042EF00F004012351010A000101E009D0CA
:1006D00004011C5100019BDF9D9804011A81BA841A
:1006E00000019E9842EF00F0040EEA6E380EE96EAB
:1006F000EF500DE0090E016E006A002EFED7012EAC
:10070000FBD78F0E006E002EFED7EF2EF3D7120010
:10071000080E0401596F829459515907000A0EE0DE
:1007200058AF02D0010E01D0000EE8A0829AE8B0C6
:10073000828A8296D89058378286EED782840001CA
:100740001200080E0401596F828459515907000A9A
:100750000EE058AF02D0010E01D0000EE8A0829A40
:10076000E8B0828A8296D89058378286EED7828403
:10077000000112000401386B385108081CE3B00E68
:1007800038253A6F586F0001C3DF100E0401586F0F
:100790000001BEDF0401586B0001BADF0401396BB0
:1007A0003951830806E3586B0001CBDF0401392B74
:1007B000F7D7382BE1D7000121EF04F08292829421
:1007C0008296829A8292140E0401386F00018CDFA7
:1007D0008282A00E0401586F00019ADFC80E040146
:1007E000586F000195DFA20E0401586F000190DFE1
:1007F0002C0E0401586F00018BDF140E0401386FBA
:10080000000172DF2E0E0401586F000181DF2F0EF0
:100810000401586F00017CDF260E0401586F0001AF
:1008200077DF810E0401586F000172DF0D0E0401A5
:10083000586F00016DDF0A0E0401386F000154DFAC
:1008400099D70A0E0401386F00014EDFC80E04016B
:10085000586F00015DDF0A0E0401386F000144DFAC
:10086000AF0E0401586F000153DF4FEF04F0100E7C
:10087000926EF30E936E810E946E896A8A6A8B6A09
:10088000280E0401386F00012FDF609060926094A1
:100890008084640E0401386F000126DF8FD7320E8A
:1008A0000401386F000120DF0401246B1A91829843
:1008B000AB88370ECD6ECC6A780E0509BA6EC00EC5
:1008C000BB6E9D809D82F212640E386F00010CDFBA
:1008D00012EF07F004016E517003F3CF01F0F4CF73
:1008E00000F07103F35000266F517003F3500020A5
:1008F000026E00011200040169316B6F6B336B33C0
:100900001F0E6B176951070B6C6F036A6C51000166
:1009100063DEE8CF6DF404016A531DE06F6B6BC4B6
:100920006EF4716B800E706F0001D4DF02C06FF443
:1009300001C06EF4040168510124016E000E022012
:10094000036E01501A0FE96E000E0320EA6EEF509D
:100950006D11EF6E1BD06F6B6BC46EF4716B800EFC
:10096000706F0001B7DF01C06EF40401685101240B
:10097000016E000E0220036E01501A0FE96E000E88
:100980000320EA6E6D51FF0AEF14EF6E00011200B2
:1009900052C4EAFF040151C4E9FFEF52D8B442D176
:1009A00052C403F05151E96E03C0EAFFEF50E50A6B
:1009B000000115E0010A1CE0120A23E0330A2AE0D4
:1009C000010A31E0120A38E0D00A3FE0030A46E0AB
:1009D0007B0A4DE0010A54E0A00A5BE062D052C4F9
:1009E000EAFF040151C4E9FF7F0EEF6E000159D008
:1009F00052C4EAFF040151C4E9FF800EEF6E00010A
:100A000050D052C4EAFF040151C4E9FF810EEF6ED9
:100A1000000147D052C4EAFF040151C4E9FF820E2D
:100A2000EF6E00013ED052C4EAFF040151C4E9FF59
:100A3000830EEF6E000135D052C4EAFF040151C4A9
:100A4000E9FF840EEF6E00012CD052C4EAFF0401CE
:100A500051C4E9FF850EEF6E000123D052C4EAFFB6
:100A6000040151C4E9FF860EEF6E00011AD052C492
:100A7000EAFF040151C4E9FF870EEF6E000111D0B7
:100A800052C4EAFF040151C4E9FF880EEF6E000171
:100A900008D052C4EAFF040151C4E9FF890EEF6E89
:100AA000000152C4EAFF040151C4E9FFEF502008DD
:100AB00007E352C4EAFF51C4E9FFEF50890830E36D
:100AC00052C403F051C4E9FF03C0EAFF200EEF5CFB
:100AD000666F6F6B6E6F716B0C0E706F0001FADEDC
:100AE00002C066F4040101C065F4040EEA6E590EFA
:100AF000E96E02C0F7FF01C069F4010E026E0C0E30
:100B0000016E6951000169EC00F00A000900EF6A0A
:100B1000F5CFEEFF012EFAD7022EF8D717D0040139
:100B2000040EEA6E590EE96E010E026E0C0E016E95
:100B3000F76A000E000169EC00F00A000900EF6A94
:100B4000F5CFEEFF012EFAD7022EF8D7080E0401DA
:100B5000556F555361E0566B56510B0858E3036AC5
:100B60005651590FE96E040E0320EA6EEFCF00F0E4
:100B7000010E555D666F6651016E04E0D89000323B
:100B8000012EFCD700A01ED0576B5351575D19E2C0
:100B9000586B5351585D13E257514F25656F5651AD
:100BA0005303F35050255825666F65C468F4696F88
:100BB00054C46AF400019FDE0401582BEAD7572B76
:100BC000E4D723D0576B5351575D1FE2586B5351F5
:100BD000585D19E257514F25656F56515303F35035
:100BE00050255825666F545302E0000E01D0010EC7
:100BF000676F65C468F466C469F46A6F00017BDEE0
:100C00000401582BE4D7572BDED7562BA5D75551C7
:100C1000550753514F279DD7512BD8B4522B000164
:100C2000B7D604010001E6EF06F004014F31536F1F
:100C3000533353331F0E53175031546F54335433BF
:100C40001F0E541753C451F45151545D37E3B00E85
:100C50005125576F586F00015BDD100E0401586F6E
:100C6000000156DD0401586B000152DD04016F6B79
:100C700051C46EF4716B800E706F00012BDE01C0E9
:100C800057F41A0E04010124016E000E022001C067
:100C900055F4566F526B52517F080EE356C4EAFF6B
:100CA0005551552BD8B4562BE96EEFCF58F40001AF
:100CB00048DD0401522BEFD7512BC6D70001EFEFCF
:100CC00006F004013C813951010A000107E0030AE2
:100CD00009E0010A0BE0070A0DE011D0050E04013E
:100CE0003B6F0ED0130E04013B6F0AD0210E04019E
:100CF0003B6F06D02F0E04013B6F02D000010401B0
:100D00003A6B3A510F083EE3036A3A513D0F016EC8
:100D1000040E032203C04FF4020E3A25036A260F85
:100D2000E96E040E0320EA6EEFCF50F44FC4EAFFE1
:100D300001C0E9FF50C4EFFF3B512F0820E1036AD7
:100D40003A513D0FE96E040E0320EA6EEF507E0823
:100D500014E0036A3A513D0FE96E040E0320EA6E77
:100D6000EF507F080AE0036A3A513D0FE96E040E26
:100D70000320EA6EEF50060801E13C9101D03C816E
:100D80003A2BBFD74D6B3CB110D07B0E3D6F7D0E23
:100D9000406F7B0E416F7D0E446F7B0E456F7D0E65
:100DA000486F7B0E496F7D0E4C6F000E3CB1010EFB
:100DB0004E6F4F6B3BC450F4040E526F3D0E516F9B
:100DC000010E536F4EC454F40001E2D50C0E040121
:100DD0003B254E6F3BC44FF4506F000126D755EFB3
:100DE00007F0F86AD09E078E360E006E100E016E68
:100DF000020EE96E000EEA6EEE6A002EFDD7012E9D
:100E0000FBD7196AB896170EAF6EA20EAC6E900E95
:100E1000AB6E0F01386B396B3A6B776A786A796A17
:100E2000000125D59D8AC80E0401386F00015CDCE5
:100E300004011AA13ED01A91000E81B8010E800D56
:100E4000F3CF38F4000E81BA010E400DF35038276D
:100E5000000E80B8010E200DF3503827000E81B02F
:100E6000010E100DF3503827000E81B2010E080D4F
:100E7000F3503827000E82B0010E040DF3503825D0
:100E8000FF0A006E00301B6F1B333F0E1B171BC485
:100E90001CF4030E275D006E003A0F0E0016005082
:100EA000010F386F396F00010CD704011AA301D06C
:060EB0001A93BFD70300F6
:0200000400F00A
:1000000000000000000000000000000000000000F0
:1000100000000000000000000000000000000000E0
:1000200000000000000000000000000000000000D0
:1000300000000000000000000000000000000000C0
:1000400000000000000000000000000000000000B0
:1000500000000000000000000000000000000000A0
:100060000000000000000000000000000000000090
:100070000000000000000000000000000000000080
:020000040030CA
:0E00000000F31E3F00BF810000800FE00F40A4
:00000001FF
